:03800000028140BA
:06800B00438CDC05083285
:20802B00C0D0C0E0C3E50933F509E50A33F50A9297E50992E0F509C3E50B33F50BE50C3371
:0F804B00F50C9296E50B92E0F50BD0E0D0D03219
:1E810000FDFF00000000000000000000000000000000000000000000FFFFFFFF7200F7
:2081400075811790F000E4F0438901D2AFD2A9D28C75C90075CBFC75CA6575C844D2AD1267
:20816000816502195412839312825F1282DE0281652205810581740075F00078FD12853FE3
:20818000F608A6F078FD12853FE60886F078F912853F86030886041285B845F070030281C0
:2081A000BC801678FD12853FE60886F012859E18F608A6F01285A780CB0281A31581158102
:2081C00022128393D293C2B5740A75F000C0E0C0F0128172158115817400F510E51075F042
:2081E000007B057C001285EB45F0700302825C8008E51004F5101480E37400F50FE50F759B
:20820000F0007B087C001285EB45F0700302824A8008E50F04F50F1480E3C2B5740375F029
:2082200000C0E0C0F012817215811581D2B5740375F000C0E0C0F012817215811581D2B453
:20824000E511A2B413F511028212E51079137A0075F000128561E511F70281F1C2932212E1
:208260008393D293C2B5740A75F000C0E0C0F0128172158115817400F50FE50F75F0007B5C
:20828000287C001285EB45F070030282DB8008E50F04F50F1480E3C2B5740375F000C0E0C3
:2082A000C0F012817215811581D2B5740375F000C0E0C0F012817215811581D2B4A2B4E538
:2082C0001713F517E51613F516E51513F515E51413F514E51313F51302828FC293227453BF
:2082E00075F086C0E0C0F0740075F00079137A00128561E775F000C0E0C0F0740275F000F5
:2083000012837F1581158115811581740075F00079137A00128561E775F0007B037C0012C2
:208320008568F512E512240AF5127400F50FE50F75F000AB127C001285EB45F07003028364
:208340005E8008E50F04F50F1480E3742075F000C0E0C0F01283A91581158102834374785D
:2083600075F000C0E0C0F01283A915811581740D75F000C0E0C0F01283A9158115812223F9
:20838000F42581F81286291283D11286290283A0D2AF22C2AF2278FB12853F8682088683A6
:2083A000E0602D1283AFA380F778FB12853FE63099FDC299F599B40A17740D80F2E43098A0
:2083C0000C3098FDC298E599B40D02740A75F00022128518868208868308E4FEFFE0700625
:2083E000128518E4F022B42551A3E0B42D05430780A3E0B4300343074024D0B40A00500B7A
:20840000CE75F00AA42EFEA3E080EEE0B46413E60886F030F7084307201285AEA6F018F66D
:208420008003B4750543070A8021B478054307108019B46F104307088011128518F0A31208
:208440008518A38095B462624307027A00C004C005C006C007AB0753031F7C00E60886F06C
:20846000128568A6F018F6EDD007D006D005D0042430B43A0040022407C0E00AE645F07032
:20848000CC128518A902EF30E505742DF0A30A128521D0E0F0A3D9FA0808EF30E7A1EAC33D
:2084A0009E509C7420F0A30A80F4B4630DAA01128518128521E6F0A380DEB47331C082C026
:2084C0008386820886837A00E06004A30A80F98683188682128518128521128518E0A31248
:2084E00085186004F0A380F2D005D00480AAB4691B86017A00E76004090A80F912851812D2
:2085000085218601E76091F009A380F8F97A01128518128521E9809ECDC583CDCCC582CC9F
:2085200022EE601A8FF020F715C002EAC39E500C742030F6027430F0A30A80EFD00222C875
:208540002581C822C92581C97A0022D083D082CF2581F581CFC082C08322CF2581F581CFF7
:208560002229F9E5F03AFA22C002C001AAF0F97E007D007F11C3E933F9EA33FADF08F5F030
:20858000E9D001D00222ED33FDEE33FEC3ED9BF5F0EE9C40E0ADF0FED380DB12859E0470A5
:2085A0000205F0221285A714B4FF0215F0221285A7F4C5F0F4C5F02212860B4029801E1206
:2085C000860B40227017801E12860B40107017800C12860B5010800512861F6009E4F5F00C
:2085E0002212861F60F7E4F5F0042212861F40F680EB12861F40EF70E480EB12861F40DD8B
:2086000070E480D912861F50DD80D2C39BC5F09C20E70720D207C345F02220D2F9D322C502
:20862000F0C39C7003E5F09B2290F000E0A360F8E0FFA3E0A3CF2582F582EF3583F58380FA
:19864000EBFBE0CB22FCE0FBA3E0CC22FAE0F9A3E0CA22253033750A00DD
:00000001FF
